:100000007A807B00DBFEDAFA758108748990F80348
:10001000F0E490F800F0748090FC03F0C295C29672
:100020007A0C7B0312074E120928758920759852A5
:10003000758DFDD28E1209D378087A74760008DAAD
:10004000FB12051A90005712052712053F1205965C
:100050007A0F1204D58028202020414E542D43359C
:10006000314D20426F6172642020202053656C6600
:100070002D74657374202050726F6772616D2090CB
:1000800001B812053390F802E0F45470B400059002
:1000900001188033B4100590012C802BB4200590FA
:1000A00001408023B43005900154801BB44005907A
:1000B00001688013B4500590017C800BB4600590FA
:1000C000019080039001A412053912053F90F802B7
:1000D000E0F420E70280AEC0E09001CC12053312BC
:1000E000053F7A051204D5D0E05470B40003020134
:1000F000E0B4100302022BB42003020284B43003E4
:100100000202A8B440030202C5B4500302034BB478
:1001100060030203DE020415544553543E204C4351
:10012000442C4C45442C534F554E44205445535475
:100130003E20383235352C444953504C415920200B
:10014000544553543E204B4559203378342C347851
:1001500038202020544553543E204F50544F2C52A9
:10016000454C4159203C2D3E544553543E20445368
:10017000313230322C4453313632302054455354CE
:100180003E2052414D2C32323233202D2D2D2D2048
:10019000544553543E2052533233322C3438352098
:1001A0003C2D2D3E544553543E204241434B555027
:1001B0002C4C422C57442020444950535720312D79
:1001C000333D4D6F646520343D52756E2A2A2A2ACC
:1001D0002020576F726B696E6720202A2A2A2A20F6
:1001E0007F087E3175F01112022112053FE5F054AF
:1001F000F090F801F0E5F023F5F012058F7A051282
:1002000004D50EDFE27EFF12022112053F74F0904A
:10021000F801F07A141204D5740090F801F002008D
:100220007F7A287821EEF608DAFC2290FC037480AD
:10023000F012023702007F75730275741290027219
:10024000858371858272857183857282E493A3852B
:1002500083718582727C0390FC00F0A3DCFC7A0839
:100260007869F608DAFC7A20120628D574D8D57396
:10027000C922010204081020408000FF00FF00AAEC
:1002800055AA55001205A4D2011205AEC201B4FF51
:1002900002800A1206378A478B4812053F90F802FF
:1002A000E0F420E7E202007F20B20775472AC2B3DC
:1002B0008005754720D2B312053F90F802E0F42084
:1002C000E7E602007F757531757612757796757859
:1002D00023757959757A55757B011206EB7AEE1202
:1002E000073A1206C0E5751206378A358B36753720
:1002F0002FE5761206378A388B39753A2FE5771253
:1003000006378A3B8B3C753D20E5781206378A3EDE
:100310008B3F75403AE5791206378A418B42754327
:100320003AE57A1206378A448B457546207AAA1236
:1003300007BD120722EB1206378A478B4812053F8A
:1003400090F802E0F420E79502007F7571807572E5
:10035000007573F77574FF1208317A20784974417B
:10036000F60804DAFB1208A675445775455275461F
:100370004975475412053F7A051204D51208EF75E6
:10038000444375454875464375474B12053F7A050A
:100390001204D57A20784975F041E6B5F01B0805BE
:1003A000F0DAF77544507545417546537547531259
:1003B000053F7A051204D580177544457545527579
:1003C000465275472112053F7A051204D512059D44
:1003D00090F802E0F420E70302007F02034B75F07F
:1003E000301209D0E5F01209357A051204D505F06E
:1003F000E5F0B43A0375F03020980B90F802E0F481
:1004000020E7E102007F12097A1206378A468B47FD
:1004100012053F80E6120596900499120533900468
:10042000AD120539908000E0B4550DA3E0B4AA08E0
:1004300075254F75264B80109080007455F0A3747D
:10044000AAF07525577526521208EFE549B4550DE7
:10045000E54AB4AA08752D4F752E4B800F75495586
:10046000754AAA1208A6752D57752E527A0A1204DB
:10047000D575344820B50375344C12053FB29790BA
:10048000F802E0F420E7EA9004C112053912053FB2
:100490007A021204D5B29780FE52414D3D78782001
:1004A000323232333D7878204241543D78456E6196
:1004B000626C6520574420262044495034206F66E2
:1004C000665761697421205761746368646F67209F
:1004D00052657365747BB37C00DCFE0000DBF8DAE8
:1004E000F4227CE60000DCFCDBF8EAB40001221A0E
:1004F00080F0C083C08290FA00F090FA01E020E71B
:10050000FCD082D08322C083C08290FA02F090FA9D
:1005100001E020E7FCD082D08322743891F2740E7F
:1005200091F2740191F2227A287821E493F6A308DB
:10053000DAF9227A14782180F27A14783580EC780E
:1005400021748012054C74C012054C2291F27A1469
:10055000E6B10608DAFA227D007C80120562BD0150
:10056000FA2290F801E0D2E3F012057790F801E06A
:10057000C2E3F012057722EA12057F1470FA22DC3A
:10058000067C80DB027D01227A507B15B157227AEE
:10059000307B15B157227A107B40B157227A907B7D
:1005A00090B157227A087869760008DAFB227C0835
:1005B0007D087E007F691205EC90F802E0540FB4CC
:1005C0000F0CDD02C200DCEE3001E374FF22C44EEA
:1005D0002000F3D200FA7B1F900608E493C39A60D0
:1005E00003A3DBF7EBC0E0B188D0E02290F801E094
:1005F00054F84EF0EFF8E690F800F07A047B00DB58
:10060000FEDAFAE4F00E0F22E8E7E6E5D8D7D6D511
:10061000B8B7B6B578777675E4E3E2E1D4D3D2D152
:10062000B4B3B2B174737271EAF97C087E007F6969
:10063000B1ECDCFCD9F422C0E0C4120645FAD0E0EB
:10064000120645FB22540FB40A0050034430229492
:1006500009444022EA120660C4FAEB1206604A22FC
:10066000B4410040022409540F22C2951206BBD2A5
:10067000961206BBEA1206A97C08E4C2951206BBD4
:10068000A29413D2951206BBDCF1FBC2961206BBF4
:1006900022C2951206BBD2961206BBEA1206A9EB3D
:1006A0001206A9C2961206BB227C08139294D29518
:1006B0001206BBC2951206BBDCF1227D04DDFE22D0
:1006C0007A87D16A8B757A89D16A8B767A8DD16A6D
:1006D0008B777A8BD16A8B7B7A85D16A8B787A8398
:1006E000D16A8B797A81D16A8B7A227A8E7B00D11A
:1006F000917A86AB75D1917A88AB76D1917A8CABB1
:1007000077D1917A8AAB7BD1917A84AB78D1917A87
:1007100082AB79D1917A80AB7AD1917A8E7B80D17C
:100720009122EB30E001227F00C3EC1350027F01E5
:10073000F5827583001207E8EF22C29212079BD25E
:100740009312079BEA120788C29312079B22C29258
:1007500012079BD29312079BEA120788EB120788B5
:10076000C29312079B1207A022C29212079BD29338
:1007700012079BEA120788EC120788EB120788C25F
:100780009312079B1207A0227D0813929100D29228
:1007900012079BC29212079BDDF0227E04DEFE222E
:1007A0007D407E00DEFEDDFA22C292F19BD293F103
:1007B0009BEAF1881207D7FBC293F19B22C292F108
:1007C0009BD293F19BEAF1881207D7FC1207D7540A
:1007D00001FBC293F19B227D08E4C292F19BA2919E
:1007E00013D292F19BDDF322E4F9FAFB7C10E5824F
:1007F00033F582E58333F5837D037803E635E0D472
:10080000F618DDF8DCE8227C107D037801C3E613DE
:10081000C0D030E703C3943030E303C39403F60839
:10082000D0D0DDEAE58313F583E58213F582DCD9C8
:100830002285718385728275F0417A64E5F0F0E576
:1008400083B57307E582B574028007A305F0DAEC7F
:1008500080E5857183857282C083C082E58312063C
:10086000378A448B457478F546F54712053F7A0080
:100870007B0A1204E2D082D08375F0417A64E0B53D
:10088000F016E583B57307E582B574028009E4F0DC
:10089000A305F0DAE980C12212059D75464575472A
:1008A0005212053F80FE1208D61208E51208E51222
:1008B00008D61208D61208D61208D61208D67849D9
:1008C0007A207B08E61340051208E580031208D65B
:1008D000DBF308DAED2200C2907904D9FED29079D8
:1008E0001ED9FE002200C2907924D9FED290221196
:1008F000D611E511E511E511E511E511E511E578F0
:10090000497A207B0812091013DBFAF608DAF42280
:1009100000C2907903D9FED2907905D9FE00A29049
:10092000791CD9FE00D290227AC811E5DAFC7A400F
:1009300011E5DAFC223099FDC299F59922120637A9
:10094000EA3135EB313522CF2FCF313D22E58331EE
:100950003DE582313D22E493B40002A322B40D05AB
:10096000120971A3223135A380EC74203135DAFAF3
:1009700022740D3135740A3135223098FDC298E564
:100980009922317AFA317AFB120654223182CF2F22
:10099000CF223182F5833182F582228587F0B41926
:1009A00008758DFDD2F70209CCB49608758DFDC28D
:1009B000F70209CCB44806758DFA0209CCB42406B6
:1009C000758DF40209CCB41206758DE885F0872286
:0B09D000D2B4223099FD0000C2B42216
:00000001FF
